:0400000080311B2808
:10000800803101300B1D00398B1E0039091C122864
:100018002000280803191128A8030B1101308B1D93
:1000280000392700961D0039091896110900880122
:1000380084319D2C210099171917991619169911B1
:10004800991019108B0191019201200091019201E0
:100058008C0123008C0121008C0122008C012000DE
:100068008D0123008D01083021008D0022008D01B3
:1000780020008E0121008E0122008E018730210090
:100088009500083024008D0021009513240090115C
:10009800220091019301200098019C012500930101
:1000A8009A01260093019A012400950182302200CA
:1000B8009700F03021009E007D309D000B179512AF
:1000C8001515951415149511200095018B160B1113
:1000D80027009401950195158B159611DC302800A1
:1000E8009D00A030250091000C30930002309E0046
:1000F800013028009E0022000C1784317E248031B4
:100108000B302000AE003B30AF005A2380318B17F4
:10011800D82028001E1125009301220097012100F4
:100128009D018B1222000C13630000000C17843110
:100138007E2480318B16823097007D3021009D000F
:100148000C30250093002000901D8C281823803146
:1001580022008E1520002E0896228031293020009A
:10016800AD006E30AC009830AB00AB0BB928AC0BCF
:10017800B928AD0BB928C02822008E110E16200010
:100188002F089622803129302000AD006E30AC0057
:100198009830AB00AB0BCE28AC0BCE28AD0BCE28DD
:1001A800D52822000E12A72820008D1908008431B6
:1001B8005124803121082004031D362922008E1580
:1001C8000E160530FD000B30FC00F230FB00FB0B77
:1001D800EB28FC0BEB28FD0BEB28F22822008E11F4
:1001E8000E120530FD000B30FC00F230FB00FB0B5B
:1001F800FB28FC0BFB28FD0BFB28022922008E158F
:100208000E160530FD000B30FC00F230FB00FB0B36
:100218000B29FC0B0B29FD0B0B29122922008E112F
:100228000E120530FD000B30FC00F230FB00FB0B1A
:100238001B29FC0B1B29FD0B1B29222922008E15CB
:100248000E160530FD000B30FC00F230FB00FB0BF6
:100258002B29FC0B2B29FD0B2B29322922008E116F
:100268000E12080018238031A60AFB302602031854
:10027800392928001E15C830250091000530FD00D9
:100288000B30FC00F230FB00FB0B4829FC0B482923
:10029800FD0B48294F2922008C150C168C178C143D
:1002A8000C158C160330FD000630FC007730FB007F
:1002B800FB0B5C29FC0B5C29FD0B5C296400E32328
:1002C80080310330FD000630FC007730FB00FB0B6B
:1002D8006B29FC0B6B29FD0B6B2964002200F523AD
:1002E80080318C150C168C178C140C158C16033059
:1002F800FD000630FC007730FB00FB0B8129FC0B6E
:100308008129FD0B81296400E32380310330FD003E
:100318000630FC007730FB00FB0B9029FC0B902982
:10032800FD0B902964002200F523A03025009100E0
:1003380022008E1584311B2480312E0896228031AC
:100348002930FD006E30FC009830FB00FB0BAA2919
:10035800FC0BAA29FD0BAA29B12922008E110E1621
:1003680084311B2480312F08962280312930FD00EA
:100378006E30FC009830FB00FB0BC029FC0BC02939
:10038800FD0BC029C72922000E120C238031200042
:100398008D1908002008962280315130FD00DC308C
:1003A800FC003430FB00FB0BD729FC0BD729FD0BD5
:1003B800D729DE290C23803120008D190800AA01D5
:1003C800A901A708031D382A22008E1520002E082F
:1003D800962280312930FD006E30FC009830FB00F9
:1003E800FB0BF429FC0BF429FD0BF429FB29F43051
:1003F8002000A800A8080319362A8D19272AF430E6
:10040800A800A901A90A2A0803190C2AAE030D2A73
:10041800AE0AFB302E02031C132A1730AE00183028
:100428002E020318AE012E08962280311530FD00E9
:100438003730FC00CA30FB00FB0B202AFC0B202ABB
:10044800FD0B202A272A20008D1DFE2929080319C3
:10045800FE29A9012A080319332AAA01FE29AA019B
:10046800AA0AFE2922008E112000270B8B2A2200BF
:100478000E1620002F08962280312930FD006E309C
:10048800FC009830FB00FB0B472AFC0B472AFD0BAE
:10049800472A4E2AF4302000A800A8080319892A00
:1004A8008D197A2AF430A800A901A90A2A08031983
:1004B8005F2AAF03602AAF0AFB302F02031C662AAB
:1004C8003B30AF003C302F020318AF012F089622B3
:1004D80080311530FD003730FC00CA30FB00FB0BC3
:1004E800732AFC0B732AFD0B732A7A2A20008D1DB0
:1004F800512A29080319512AA9012A080319862A09
:10050800AA01512AAA01AA0A512A22000E12200081
:1005180027080319912AA701932AA701A70A5A2392
:1005280080310C2BF7000C23803128001E150A306F
:10053800F0007708AA238031F5000A30F000770828
:10054800C2238031F600BA2A22008C15EC2A220038
:100558000C16EC2A22008C17EC2A22008C14EC2AA8
:1005680022000C15EC2A22008C16EC2A7508003A99
:100578000319A82A013A0319AB2A033A0319AE2A28
:10058800013A0319B12A073A0319B42A013A03199F
:10059800B72AEC2A22008E17080022000D15080041
:1005A80022000E17080022008D16080022000D16E2
:1005B800080022000D17080022008D1708002200ED
:1005C8008D14080022008E16080022000D14080061
:1005D8007608003A0319CE2A013A0319D12A033AB8
:1005E8000319D42A013A0319D72A073A0319DA2A30
:1005F800013A0319DD2A033A0319E02A013A0319DB
:10060800E32A0F3A0319E62A013A031D0800E92AEA
:1006180028001E1122000E118C110C128C138C1044
:100628000C118C12F5230800013045232000B0007E
:100638000F39F5000A30F000300E0F3984314524A7
:1006480080317507B000023045232000AF000F3914
:10065800F5000A30F0002F0E0F398431452480311F
:100668007507AF00033045232000AE000F39F500B1
:100678000A30F0002E0E0F39843145247507AE007C
:100688000800F30084318C248031D0308C238031F1
:1006980073088C2384318C248031D1308C238031B1
:1006A8000024F400843198247408080084318C24D0
:1006B8008031D0308C23803100308C238031003061
:1006C8008C23803100308C2380310A30F0002000E8
:1006D8002F08C2238031F5000A30F0002F08AA2322
:1006E8008031890EF03975078C2380310A30F0008B
:1006F80020002E08C2238031F5000A30F0002E08B1
:10070800AA238031890EF03975078C238431982CFF
:10071800F1000830F200F2080319A42BF203710863
:10072800F000720A982BF036890B972B701C9F2BC0
:1007380022008E14A12B22008E10DA2380318F2BF9
:1007480021008E14DA2321008E100800F100F30135
:1007580070080319C02BF201F20AF01BB52BF03513
:10076800B02BF33570087102031CBD2B7008F10221
:100778007314F036F20BB52B73080800F20008303A
:10078800F300F4017208F1000730F136890BC92B28
:1007980074357104F400F23570087402031CD62B0A
:1007A8007008F402F30BC62B7408080084319524F2
:1007B800803122000E14843195240E100800220086
:1007C8008C110C128C138C100C118C128E170D15A9
:1007D8000E178D160D160D178D178D148E160D14F8
:1007E80008008E130D110E138D120D120D138D139B
:1007F8008D108E120D100800F1010830F2008E14D1
:10080800F2080319172CF20320008E1C142C013057
:10081800F000720A102CF035890B0F2C7008F104C7
:10082800DA238031042C21008E107108080008306A
:100838002000A2002000A20803190800A203A40AAD
:10084800063024020318A401A50A0A302502031859
:10085800A5010A30F000240845242507A300230831
:100868008231962284310230FA003730F900AC30F8
:10087800F800F80B3D2CF90B3D2CFA0B3D2C442CC1
:100888001E2CF200F10170087218F107F035F236EB
:10089800F208031D472C7108080021009D149D18BB
:1008A800532C1C082000A000A101A100A0012100D8
:1008B8001B082000A004023021025930031920022D
:1008C800031C692CA001A10108005830F000023077
:1008D800F10020087002A0002108713BA10000303F
:1008E8002102333003192002031C08003230A00013
:1008F800A10108008C24D03083318C2384310C3042
:1009080083318C2384313F3083318C238431982C7C
:1009180022008E140E14952484318E1095240E1006
:10092800080000000000080022000E1495248E1410
:100938000800A001A101A201A301A401A501A6012B
:10094800A701A8011730AE003B30AF001E30B00041
:06095800200080311E2882
:020000040001F9
:04000E0084D9FFDDB5
:10E000000000730000000000FF00FF00FF00FF00A1
:00000001FF
